:10000000C828A2008417800484138E010C1C8E0063
:1000100023200319C32823200319C3282320C3281E
:10002000A20059200C080D040319C328BD20841315
:100030002208800664001C281D288C0A03198D0FD5
:100040001A288006C32822088E0601308C008D01F4
:10005000000822050E06031D08008C0A03198D0FE7
:10006000282808008F002408840022095A208413BD
:100070008F080319C328F03091000E0880389000D3
:10008000F03091030319910003198F030319C3285A
:1000900049285D2003010C1822088E1F22088E08B3
:1000A00003190301900F562880063D2857280000A9
:1000B0004028FF3A84178005C3280D080C04031953
:1000C0008C0A80300C1A8D060C198D068C188D0642
:1000D0000D0D8C0D8D0DC3288F018E00FF308E0706
:1000E000031C8F07031CC32803308D00DF307A20E8
:1000F0006E288D01E83E8C008D09FC30031C83289E
:100100008C07031880288C0764008D0F80280C183A
:1001100089288C1C8D2800008D2808008E00013055
:10012000912894000F080D02031D98280E080C0258
:10013000043003180130031902301405031DFF3089
:10014000C32891019001103092000D0D900D910D7A
:100150000E0890020F08031C0F0F91020318B72816
:100160000E0890070F0803180F0F910703108C0D4E
:100170008D0D920BA5280C08C3288C098D098C0ABB
:1001800003198D0A08008313031383126400080007
:100190008316850108308600831206118316061126
:1001A000831206108316061083128610831686109B
:1001B00083120F212C088C002D088D008F012F3009
:1001C0008E20031DD9280630A4001030A200503024
:1001D0002C079E002D080318013E9F001E088E006C
:1001E0000A30322028088C0029088D008F01053044
:1001F0008E20031D0429061483160610831286140C
:100200008316861083120C2906108316061083129B
:100210008610831686108312D92863000D290130B9
:100220008C008D01063084000430102001308C00D9
:1002300006308400083001200C08AA000D08AB002D
:100240002A088C002B088D000F308E008F01A12012
:10025000A8000D08A9002A088C002B088D00063084
:100260008E008F01A120AC000D08AD0001306C2084
:02027000080084
:02400E00F53F7C
:00000001FF
